 gptsdk

 Timestamp is 4fb05c80 (Mon May 14 13:14:40 2012)

 Preferred load address is 10000000

 Start         Length     Name                   Class
 0001:00000000 00000004H .CRT$XCA                CODE
 0001:00000004 00000004H .CRT$XCZ                CODE
 0001:00000008 00000004H .CRT$XIA                CODE
 0001:0000000c 00000004H .CRT$XIZ                CODE
 0001:00000010 00000004H .CRT$XPA                CODE
 0001:00000014 00000004H .CRT$XPZ                CODE
 0001:00000018 00000004H .CRT$XTA                CODE
 0001:0000001c 00000004H .CRT$XTZ                CODE
 0001:00000020 00000560H .rdata                  CODE
 0001:00000580 00000023H .rdata$debug            CODE
 0001:000005a4 000011fcH .text                   CODE
 0001:000017a0 00000014H .xdata                  CODE
 0001:000017b4 00000014H .idata$2                CODE
 0001:000017c8 00000014H .idata$3                CODE
 0001:000017dc 00000058H .idata$4                CODE
 0001:00001834 0000000cH .idata$6                CODE
 0001:00001840 0000012bH .edata                  CODE
 0002:00000000 00000058H .idata$5                DATA
 0002:00000058 0000044cH .data                   DATA
 0002:000004a4 00000010H .bss                    DATA
 0003:00000000 000000d8H .pdata                  DATA

  Address         Publics by Value              Rva+Base       Lib:Object

 0000:00000000       ___safe_se_handler_count   00000000     <absolute>
 0000:00000000       ___safe_se_handler_table   00000000     <absolute>
 0001:00000000       __xc_a                     10001000     corelib0:crt0init.obj
 0001:00000004       __xc_z                     10001004     corelib0:crt0init.obj
 0001:00000008       __xi_a                     10001008     corelib0:crt0init.obj
 0001:0000000c       __xi_z                     1000100c     corelib0:crt0init.obj
 0001:00000010       __xp_a                     10001010     corelib0:crt0init.obj
 0001:00000014       __xp_z                     10001014     corelib0:crt0init.obj
 0001:00000018       __xt_a                     10001018     corelib0:crt0init.obj
 0001:0000001c       __xt_z                     1000101c     corelib0:crt0init.obj
 0001:0000003c       ??_C@_1O@IKMMPJPA@?$AA?9?$AA?9?$AA?$CF?$AAs?$AA?$AN?$AA?6?$AA?$AA@ 1000103c     gptsdk_common_topaz_v1:gptsdk.obj
 0001:0000004c       ??_C@_1DM@FDLDNGJJ@?$AA?$CF?$AAs?$AA?3?$AA?5?$AA?5?$AAC?$AAr?$AAe?$AAa?$AAt?$AAe?$AAF?$AAi?$AAl?$AAe?$AA?5?$AAG?$AAP?$AAT?$AA?5?$AAf?$AAa?$AAi?$AAl?$AAe?$AAd?$AA?$CB?$AA?$AN?$AA?6?$AA?$AA@ 1000104c     gptsdk_common_topaz_v1:gptsdk.obj
 0001:00000088       ??_C@_1O@JNDDBHKG@?$AA?$CL?$AA?$CL?$AA?$CF?$AAs?$AA?$AN?$AA?6?$AA?$AA@ 10001088     gptsdk_common_topaz_v1:gptsdk.obj
 0001:00000098       ??_C@_1BM@NDHBHMFE@?$AAG?$AAp?$AAt?$AAO?$AAp?$AAe?$AAn?$AAH?$AAa?$AAn?$AAd?$AAl?$AAe?$AA?$AA@ 10001098     gptsdk_common_topaz_v1:gptsdk.obj
 0001:000000b4       ??_C@_1DE@BBBAGJCD@?$AA?$CF?$AAs?$AA?3?$AA?5?$AAC?$AAl?$AAo?$AAs?$AAe?$AAH?$AAa?$AAn?$AAd?$AAl?$AAe?$AA?5?$AAf?$AAa?$AAi?$AAl?$AAe?$AAd?$AA?$CB?$AA?$AN?$AA?6?$AA?$AA@ 100010b4     gptsdk_common_topaz_v1:gptsdk.obj
 0001:000000e8       ??_C@_1BO@BKIEOEBD@?$AAG?$AAp?$AAt?$AAC?$AAl?$AAo?$AAs?$AAe?$AAH?$AAa?$AAn?$AAd?$AAl?$AAe?$AA?$AA@ 100010e8     gptsdk_common_topaz_v1:gptsdk.obj
 0001:00000108       ??_C@_1FG@EJIBPPCL@?$AA?$CF?$AAs?$AA?3?$AA?5?$AAG?$AAP?$AAT?$AA_?$AAI?$AAO?$AAC?$AAT?$AAL?$AA_?$AAT?$AAI?$AAM?$AAE?$AAR?$AA_?$AAC?$AAR?$AAE?$AAA?$AAT?$AAE?$AA_?$AAE?$AAV?$AAE?$AAN?$AAT@ 10001108     gptsdk_common_topaz_v1:gptsdk.obj
 0001:00000160       ??_C@_1DC@BGIPIMAG@?$AA?$CF?$AAs?$AA?3?$AA?5?$AAC?$AAr?$AAe?$AAa?$AAt?$AAe?$AAE?$AAv?$AAe?$AAn?$AAt?$AA?5?$AAf?$AAa?$AAi?$AAl?$AAe?$AAd?$AA?$AN?$AA?6?$AA?$AA@ 10001160     gptsdk_common_topaz_v1:gptsdk.obj
 0001:00000194       ??_C@_1CI@GJDHBDMJ@?$AAG?$AAp?$AAt?$AAC?$AAr?$AAe?$AAa?$AAt?$AAe?$AAT?$AAi?$AAm?$AAe?$AAr?$AAE?$AAv?$AAe?$AAn?$AAt?$AA?$AA@ 10001194     gptsdk_common_topaz_v1:gptsdk.obj
 0001:000001c0       ??_C@_1FI@EPDMKDJI@?$AA?$CF?$AAs?$AA?3?$AA?5?$AAG?$AAP?$AAT?$AA_?$AAI?$AAO?$AAC?$AAT?$AAL?$AA_?$AAT?$AAI?$AAM?$AAE?$AAR?$AA_?$AAR?$AAE?$AAL?$AAE?$AAA?$AAS?$AAE?$AA_?$AAE?$AAV?$AAE?$AAN@ 100011c0     gptsdk_common_topaz_v1:gptsdk.obj
 0001:00000218       ??_C@_1CK@LBGFOLDP@?$AAG?$AAp?$AAt?$AAR?$AAe?$AAl?$AAe?$AAa?$AAs?$AAe?$AAT?$AAi?$AAm?$AAe?$AAr?$AAE?$AAv?$AAe?$AAn?$AAt?$AA?$AA@ 10001218     gptsdk_common_topaz_v1:gptsdk.obj
 0001:00000248       ??_C@_1FE@GMIEINBJ@?$AA?$CF?$AAs?$AA?3?$AA?5?$AAG?$AAP?$AAT?$AA_?$AAI?$AAO?$AAC?$AAT?$AAL?$AA_?$AAT?$AAI?$AAM?$AAE?$AAR?$AA_?$AAS?$AAH?$AAO?$AAW?$AA_?$AAC?$AAL?$AAK?$AAS?$AAR?$AAC?$AA?5@ 10001248     gptsdk_common_topaz_v1:gptsdk.obj
 0001:0000029c       ??_C@_1CA@HEKLAELP@?$AAG?$AAp?$AAt?$AAS?$AAh?$AAo?$AAw?$AAT?$AAi?$AAm?$AAe?$AAr?$AAS?$AAr?$AAc?$AA?$AA@ 1000129c     gptsdk_common_topaz_v1:gptsdk.obj
 0001:000002c0       ??_C@_1EI@EPCHCPAF@?$AA?$CF?$AAs?$AA?3?$AA?5?$AAG?$AAP?$AAT?$AA_?$AAI?$AAO?$AAC?$AAT?$AAL?$AA_?$AAT?$AAI?$AAM?$AAE?$AAR?$AA_?$AAS?$AAT?$AAA?$AAR?$AAT?$AA?5?$AAf?$AAa?$AAi?$AAl?$AAe?$AAd@ 100012c0     gptsdk_common_topaz_v1:gptsdk.obj
 0001:00000308       ??_C@_1BC@OFFDFDML@?$AAG?$AAp?$AAt?$AAS?$AAt?$AAa?$AAr?$AAt?$AA?$AA@ 10001308     gptsdk_common_topaz_v1:gptsdk.obj
 0001:00000320       ??_C@_1EG@BILHNAEH@?$AA?$CF?$AAs?$AA?3?$AA?5?$AAG?$AAP?$AAT?$AA_?$AAI?$AAO?$AAC?$AAT?$AAL?$AA_?$AAT?$AAI?$AAM?$AAE?$AAR?$AA_?$AAS?$AAT?$AAO?$AAP?$AA?5?$AAf?$AAa?$AAi?$AAl?$AAe?$AAd?$AA?$CB@ 10001320     gptsdk_common_topaz_v1:gptsdk.obj
 0001:00000368       ??_C@_1BA@OFEEAMNJ@?$AAG?$AAp?$AAt?$AAS?$AAt?$AAo?$AAp?$AA?$AA@ 10001368     gptsdk_common_topaz_v1:gptsdk.obj
 0001:00000378       ??_C@_1EK@JPDOOOCL@?$AA?$CF?$AAs?$AA?3?$AA?5?$AAG?$AAP?$AAT?$AA_?$AAI?$AAO?$AAC?$AAT?$AAL?$AA_?$AAT?$AAI?$AAM?$AAE?$AAR?$AA_?$AAR?$AAE?$AAS?$AAU?$AAM?$AAE?$AA?5?$AAf?$AAa?$AAi?$AAl?$AAe@ 10001378     gptsdk_common_topaz_v1:gptsdk.obj
 0001:000003c4       ??_C@_1BE@NBGBKHND@?$AAG?$AAp?$AAt?$AAR?$AAe?$AAs?$AAu?$AAm?$AAe?$AA?$AA@ 100013c4     gptsdk_common_topaz_v1:gptsdk.obj
 0001:000003d8       ??_C@_1FI@PBPPIGLF@?$AA?$CF?$AAs?$AA?3?$AA?5?$AAG?$AAP?$AAT?$AA_?$AAI?$AAO?$AAC?$AAT?$AAL?$AA_?$AAT?$AAI?$AAM?$AAE?$AAR?$AA_?$AAU?$AAP?$AAD?$AAA?$AAT?$AAE?$AA_?$AAP?$AAE?$AAR?$AAI?$AAO@ 100013d8     gptsdk_common_topaz_v1:gptsdk.obj
 0001:00000430       ??_C@_1CA@NCBHBOGD@?$AAG?$AAp?$AAt?$AAU?$AAp?$AAd?$AAa?$AAt?$AAe?$AAP?$AAe?$AAr?$AAi?$AAo?$AAd?$AA?$AA@ 10001430     gptsdk_common_topaz_v1:gptsdk.obj
 0001:00000450       ??_C@_1FA@KDKMGMBM@?$AA?$CF?$AAs?$AA?3?$AA?5?$AAG?$AAP?$AAT?$AA_?$AAI?$AAO?$AAC?$AAT?$AAL?$AA_?$AAT?$AAI?$AAM?$AAE?$AAR?$AA_?$AAG?$AAE?$AAT?$AA_?$AAC?$AAO?$AAU?$AAN?$AAT?$AA?5?$AAf?$AAa@ 10001450     gptsdk_common_topaz_v1:gptsdk.obj
 0001:000004a0       ??_C@_1CG@PIDCBCOB@?$AAG?$AAp?$AAt?$AAG?$AAe?$AAt?$AAC?$AAo?$AAu?$AAn?$AAt?$AAe?$AAr?$AAV?$AAa?$AAl?$AAu?$AAe?$AA?$AA@ 100014a0     gptsdk_common_topaz_v1:gptsdk.obj
 0001:000004c8       ??_C@_1FM@HGNPPPPG@?$AA?$CK?$AA?$CK?$AA?$CK?$AA?$CK?$AA?$CK?$AA?5?$AAD?$AAL?$AAL?$AA?5?$AAP?$AAR?$AAO?$AAC?$AAE?$AAS?$AAS?$AA?5?$AAD?$AAE?$AAT?$AAA?$AAC?$AAH?$AA?5?$AAF?$AAR?$AAO?$AAM?$AA?5?$AAG?$AAP@ 100014c8     gptsdk_common_topaz_v1:gptsdk.obj
 0001:00000528       ??_C@_1FI@GHBHGBCI@?$AA?$CK?$AA?$CK?$AA?$CK?$AA?$CK?$AA?$CK?$AA?5?$AAD?$AAL?$AAL?$AA?5?$AAP?$AAR?$AAO?$AAC?$AAE?$AAS?$AAS?$AA?5?$AAA?$AAT?$AAT?$AAA?$AAC?$AAH?$AA?5?$AAT?$AAO?$AA?5?$AAG?$AAP?$AAT?$AA?5@ 10001528     gptsdk_common_topaz_v1:gptsdk.obj
 0001:000005a4       GptOpenHandle              100015a4 f   gptsdk_common_topaz_v1:gptsdk.obj
 0001:000006c0       GptCloseHandle             100016c0 f   gptsdk_common_topaz_v1:gptsdk.obj
 0001:000007bc       GptCreateTimerEvent        100017bc f   gptsdk_common_topaz_v1:gptsdk.obj
 0001:0000095c       GptReleaseTimerEvent       1000195c f   gptsdk_common_topaz_v1:gptsdk.obj
 0001:00000a24       GptShowTimerSrc            10001a24 f   gptsdk_common_topaz_v1:gptsdk.obj
 0001:00000ad8       GptStart                   10001ad8 f   gptsdk_common_topaz_v1:gptsdk.obj
 0001:00000ba4       GptStop                    10001ba4 f   gptsdk_common_topaz_v1:gptsdk.obj
 0001:00000c58       GptResume                  10001c58 f   gptsdk_common_topaz_v1:gptsdk.obj
 0001:00000d0c       GptUpdatePeriod            10001d0c f   gptsdk_common_topaz_v1:gptsdk.obj
 0001:00000dc0       GptGetCounterValue         10001dc0 f   gptsdk_common_topaz_v1:gptsdk.obj
 0001:00000e74       DllEntry                   10001e74 f   gptsdk_common_topaz_v1:gptsdk.obj
 0001:00000f3c       CreateFileW                10001f3c f   coredll:COREDLL.dll
 0001:00000f4c       NKDbgPrintfW               10001f4c f   coredll:COREDLL.dll
 0001:00000f5c       CloseHandle                10001f5c f   coredll:COREDLL.dll
 0001:00000f6c       DeviceIoControl            10001f6c f   coredll:COREDLL.dll
 0001:00000f7c       CreateEventW               10001f7c f   coredll:COREDLL.dll
 0001:00000f8c       DisableThreadLibraryCalls  10001f8c f   coredll:COREDLL.dll
 0001:00000f9c       RegisterDbgZones           10001f9c f   coredll:COREDLL.dll
 0001:00000fac       _DllEntryCRTStartup        10001fac f   corelib0:pegdentry.obj
 0001:0000101c       exit                       1000201c f   corelib0:cexit.obj
 0001:0000119c       _exit                      1000219c f   corelib0:cexit.obj
 0001:000011c0       _cexit                     100021c0 f   corelib0:cexit.obj
 0001:000011dc       _c_exit                    100021dc f   corelib0:cexit.obj
 0001:000011f8       GetCurrentProcess          100021f8 f i corelib0:cexit.obj
 0001:00001210       _initterm                  10002210 f   corelib0:crt0dat.obj
 0001:00001264       _cinit                     10002264 f   corelib0:crt0dat.obj
 0001:00001298       __security_init_cookie     10002298 f   corelib0:seccinit.obj
 0001:00001368       _onexit                    10002368 f   corelib0:onexit.obj
 0001:0000166c       atexit                     1000266c f   corelib0:onexit.obj
 0001:000016c0       wcslen                     100026c0 f   corelib1:COREDLL.dll
 0001:000016d0       free                       100026d0 f   corelib1:COREDLL.dll
 0001:000016e0       __security_gen_cookie2     100026e0 f   corelib1:COREDLL.dll
 0001:000016f0       __C_specific_handler       100026f0 f   corelib1:COREDLL.dll
 0001:00001700       malloc                     10002700 f   corelib1:COREDLL.dll
 0001:00001710       realloc                    10002710 f   corelib1:COREDLL.dll
 0001:00001720       _msize                     10002720 f   corelib1:COREDLL.dll
 0001:00001730       DeleteCriticalSection      10002730 f   coredll:COREDLL.dll
 0001:00001740       InterlockedExchange        10002740 f   coredll:COREDLL.dll
 0001:00001750       TerminateProcess           10002750 f   coredll:COREDLL.dll
 0001:00001760       EnterCriticalSection       10002760 f   coredll:COREDLL.dll
 0001:00001770       InterlockedCompareExchange 10002770 f   coredll:COREDLL.dll
 0001:00001780       InitializeCriticalSection  10002780 f   coredll:COREDLL.dll
 0001:00001790       LeaveCriticalSection       10002790 f   coredll:COREDLL.dll
 0001:000017b4       __IMPORT_DESCRIPTOR_COREDLL 100027b4     coredll:COREDLL.dll
 0001:000017c8       __NULL_IMPORT_DESCRIPTOR   100027c8     coredll:COREDLL.dll
 0002:00000000       __imp_CreateFileW          10003000     coredll:COREDLL.dll
 0002:00000004       __imp_NKDbgPrintfW         10003004     coredll:COREDLL.dll
 0002:00000008       __imp_CloseHandle          10003008     coredll:COREDLL.dll
 0002:0000000c       __imp_DeviceIoControl      1000300c     coredll:COREDLL.dll
 0002:00000010       __imp_CreateEventW         10003010     coredll:COREDLL.dll
 0002:00000014       __imp_DisableThreadLibraryCalls 10003014     coredll:COREDLL.dll
 0002:00000018       __imp_RegisterDbgZones     10003018     coredll:COREDLL.dll
 0002:0000001c       __imp_wcslen               1000301c     corelib1:COREDLL.dll
 0002:00000020       __imp_free                 10003020     corelib1:COREDLL.dll
 0002:00000024       __imp___security_gen_cookie2 10003024     corelib1:COREDLL.dll
 0002:00000028       __imp___C_specific_handler 10003028     corelib1:COREDLL.dll
 0002:0000002c       __imp_malloc               1000302c     corelib1:COREDLL.dll
 0002:00000030       __imp_realloc              10003030     corelib1:COREDLL.dll
 0002:00000034       __imp__msize               10003034     corelib1:COREDLL.dll
 0002:00000038       __imp_DeleteCriticalSection 10003038     coredll:COREDLL.dll
 0002:0000003c       __imp_InterlockedExchange  1000303c     coredll:COREDLL.dll
 0002:00000040       __imp_TerminateProcess     10003040     coredll:COREDLL.dll
 0002:00000044       __imp_EnterCriticalSection 10003044     coredll:COREDLL.dll
 0002:00000048       __imp_InterlockedCompareExchange 10003048     coredll:COREDLL.dll
 0002:0000004c       __imp_InitializeCriticalSection 1000304c     coredll:COREDLL.dll
 0002:00000050       __imp_LeaveCriticalSection 10003050     coredll:COREDLL.dll
 0002:00000054       \177COREDLL_NULL_THUNK_DATA 10003054     coredll:COREDLL.dll
 0002:00000058       dpCurSettings              10003058     gptsdk_common_topaz_v1:gptsdk.obj
 0002:0000049c       __security_cookie          1000349c     corelib0:seccinit.obj
 0002:000004a0       __security_cookie_complement 100034a0     corelib0:seccinit.obj
 0002:000004a4       _exitflag                  100034a4     corelib0:cexit.obj
 0002:000004a8       __onexitend                100034a8     <common>
 0002:000004ac       __onexitbegin              100034ac     <common>
 0002:000004b0       g_pcsExit                  100034b0     <common>

 entry point at        0001:00000fac

 Static symbols

 0001:00001040       doexit                     10002040 f   corelib0:cexit.obj
 0001:000013c4       lockexit                   100023c4 f   corelib0:onexit.obj
 0001:00001460       unlockexit                 10002460 f   corelib0:onexit.obj
 0001:0000148c       _onexit_nolock             1000248c f   corelib0:onexit.obj
